:100000000C940C020C9429020C9444020C942902C6
:100010000C9429020C9429020C9429020C942902B4
:100020000C9429020C9429020C94CB210C942902E3
:100030000C9429020C9429020C9429020C94290294
:100040000C9429020C9429020C9429020C94290284
:100050000C942902530653067F067F06E706050720
:100060001D081D081007A907BA07BA0729001E00B6
:100070001F002000210022002B0014001A0008009D
:1000800015001C00015104001600070009000A00B9
:100090001D001B000600050000002C0000000000F1
:1000A0000000C45C00000000000000000000000030
:1000B0000000000000000000000000000000000040
:1000C00000000000000000000000000000047F3F6E
:1000D0001F643214643214783C1E1E140A05222355
:1000E000252628292A2C2D2F3032333536383A3B15
:1000F0003D3E4042434547494A4C4E505153555767
:10010000595A5C5E6062646668696B6D6F71737585
:1001100077797B7D7F81838587898A8C8E90929485
:1001200096989A9C9E9FA1A3A5A7A8AAACAEAFB192
:10013000B3B4B6B8B9BBBCBEBFC1C2C3C5C6C7C9DC
:10014000CACBCCCDCED0D1D2D2D3D4D5D6D7D7D896
:10015000D9D9DADADBDBDBDCDCDCDCDCDDDDDDDDE8
:10016000DCDCDCDCDCDBDBDBDADAD9D9D8D7D7D6F0
:10017000D5D4D3D2D2D1D0CECDCCCBCAC9C7C6C5A7
:10018000C3C2C1BFBEBCBBB9B8B6B4B3B1AFAEACED
:10019000AAA8A7A5A3A19F9E9C9A98969492908E98
:1001A0008C8A89878583817F7D7B79777573716F71
:1001B0006D6B6968666462605E5C5A59575553514D
:1001C000504E4C4A4947454342403E3D3B3A383603
:1001D000353332302F2D2C2A292826252322FFAA19
:1001E0007F554000010101010101010101020202EC
:1001F00002020202020203030303030303030404D3
:10020000040404040405050505050606060606079C
:100210000707070708080808090909090A0A0A0B55
:100220000B0B0C0C0C0D0D0D0E0E0E0F0F0F1010F6
:10023000111111121213131414151516161717187D
:100240001819191A1A1B1B1C1D1D1E1E1F202021E8
:100250002222232424252626272829292A2B2C2D2F
:100260002D2E2F30313232333435363738393A3B50
:100270003C3D3E3F404142434445464748494A4C45
:100280004D4E4F50515354555658595A5B5D5E5F11
:10029000616264656668696B6C6D6F7072737577A7
:1002A000787A7B7D7E8082838587888A8C8E8F9109
:1002B000939596989A9C9EA0A2A3A5A7A9ABADAF33
:1002C000B1B3B5B7BABCBEC0C2C4C6C9CBCDCFD11D
:1002D000D4D6D8DBDDDFE2E4E7E9EBEEF0F3F5F8C6
:1002E000FAFDFF09023B00020100A0FA0904000028
:1002F000010301010009210101000122400007055D
:100300008103080001090401000103000000092124
:1003100001010001227B000705830308000112018F
:10032000100100000008544B2323010001020001CA
:100330000E0341004D004100470032003300000031
:1003400016034B006F006F006C00650072007400B4
:1003500072006F006E000000040309040501090229
:10036000A10185020901A10005091901290815004B
:1003700025019508750181020501093009311581B2
:10038000257F95027508810609381581257F95011D
:1003900075088106050C0A38021581257F950175BF
:1003A000088106C0C005010980A101850319012A41
:1003B000B700150126B700950175108100C0050C26
:1003C0000901A101850419012AA002150126A00234
:1003D000950175108100C005010906A101050719E5
:1003E000E029E71500250195087501810295017541
:1003F0000881030507190029FF150026FF0095064F
:1004000075088100050819012905950575019102F6
:10041000950175039103C00011241FBECFE5D8E0FC
:10042000DEBFCDBF11E0A0E6B0E0ECE1FCE402C02D
:1004300005900D92AE31B107D9F722E0AEE1B1E0FF
:1004400001C01D92A93CB207E1F70E94FF130C9472
:100450000C260C940000A82FB92F80E090E041E01A
:1004600050EA609530E009C02D91822797958795D5
:1004700010F084279527305EC8F36F5FA8F30895C6
:10048000EADF8D939D930895CF93CFB7CF93C39514
:10049000839BE9F7839B0EC0839B0CC0839B0AC0A0
:1004A000839B08C0839B06C0C091A002C395C093E4
:1004B000A002A6C0DF93C0919F02DD27C955DD4F82
:1004C000839B02C0DF91E6CF2F930F931F9300B35E
:1004D0002FEF03FB20F94F933F9310B34FEF01270A
:1004E00003FB21F93BE031C04E7F012F10B32160A7
:1004F00028C0102F4D7F2260000000B329C04B7F21
:100500002460012F000010B32BC010B3477F286078
:100510002AC04F7E00B320612CC04F7D10B32062F3
:100520002FC04F7B00B3206432C0422700B34993F1
:100530004FEF0000102713FB20F910B31C70C9F116
:10054000297F91F2012703FB21F900B3237F89F270
:10055000315058F1102713FB22F910B3277E79F29E
:10056000012703FB23F92F7C81F200B3102713FB33
:1005700024F92F7971F200C010B3012703FB25F98C
:100580002F7359F200C000B3102713FB26F9223055
:1005900040F200C010B3012703FB27F9243028F6EE
:1005A0004F77206810B30000F9CF10E81ABF00277A
:1005B0001CC03B503195C31BD04010E81ABF0881C6
:1005C000033C11F10B3401F120919C021981110FB0
:1005D0001213EDCF4A81441F093669F10D3211F033
:1005E000013E29F74F7009F0042F0093A5023F91B7
:1005F0004F911F910F912F91DF91CAB7C7FD47CF40
:10060000CF91CFBFCF9118952091A502222379F3E6
:100610001091A302112309F044C034300AF443C0FE
:100620003093A30220939E0210919F023BE0311B66
:1006300030939F0238C00091A302013094F50AE57F
:100640004F7049F430918C0034FD2FC000938C0022
:10065000C9E7D2E02EC0433059F0443091F03091D8
:10066000840234FD22C000938402C5E8D2E021C098
:100670003091BD0234FD19C00093BD02CEEBD2E033
:1006800018C03091900234FD10C000939002C1E96F
:10069000D2E00FC02795A8F45150A9F4220F000012
:1006A000F9CF4AE503C042ED01C0432FC4E1D0E0D9
:1006B00032E011B31C60939A11BB02B320E41CE03A
:1006C0005F93012756E002BB279520F4515021F497
:1006D000220FF9CF012756E000003B5A02BBD0F2AF
:1006E000279528F4515029F4220F0000F9CF012753
:1006F00056E0279502BB20F4515021F4220FF9CF88
:10070000012756E02991332302BB21F6037F109184
:10071000A402110FC651D04002BB11F010939C02ED
:1007200010E81ABF086011B3137F402F437F5F9119
:1007300000C000C002BB11BB42BB59CF81E008958D
:1007400081E008950C94A00308950C94A4031F93D2
:10075000CF93DF9300D000D01F92CDB7DEB749838F
:100760005A836B833091210189819A81311114C0A0
:10077000662359F0222349F00E945C0A182F682F43
:1007800089819A810E94030A03C00E942F0A182FB0
:1007900069817A81812F04C00E945C0A69817A8113
:1007A0000F900F900F900F900F90DF91CF911F91AE
:1007B0000C948111FC01262F40815181628173814B
:1007C00084810C94A70381E00895CF93DF93EC011B
:1007D00060E00E94DA03BE01DF91CF910C94A50383
:1007E0000C94C4120C94C01208950E94AD080E948B
:1007F000F4032FEB87E299E0215080409040E1F72D
:1008000000C000000C94F1210F931F93CF93DF934E
:100810008C0161E00E94DA03EC01B8010E94A2039E
:10082000882309F444C0B801CE010E94A01F882388
:10083000F1F1B801CE010E94B41D8823C1F1B801C5
:10084000CE010E94FC1E882391F1B801CE010E94C6
:10085000C71C882361F1F8018281882309F1CB3517
:100860008DE5D807C1F050F4C115FCE5DF0781F034
:10087000CF3DDC45A9F40E94930F19C0CC35EDE5BE
:10088000DE0761F0CD35DD4559F40E94D60E08C073
:100890000E94F5030CC00E94DF0E02C00E94E20E0F
:1008A000C801DF91CF911F910F910C949E0380E0BE
:1008B000DF91CF911F910F9108950E9476210C94A2
:1008C00076040E9479040C947C2108950C946504AC
:1008D00081E008950C9468040895CF93C82F0E9476
:1008E00066048C2F0E946A04CF91089580E00C94D6
:1008F0006D040E94D5200C946D040E94D520909127
:100900002001891721F0809320010C946D04089533
:10091000CF93DF93CDB7DEB72B970FB6F894DEBF3A
:100920000FBECDBF4F83588769877A878B87611148
:100930000E94220E9E012F5F3F4F86E0F901119227
:100940008A95E9F785E0FE013796D90101900D926D
:100950008A95E1F789819A814C815D81452B31F03F
:100960009F3F31F491E08F3F19F403C091E001C043
:1009700090E090FF09C049815A816B817C818D8113
:100980009E810E94430D05C0C9010E94E3038111AD
:10099000F2CF2B960FB6F894DEBF0FBECDBFDF911E
:1009A000CF910895FC01808191810E949E0A089553
:1009B000CF93882309F4A4C0C82F8238C1F40E94C1
:1009C000D52081FD9DC069E3809162009091630014
:1009D0000E9468210E94440E2FE789EA93E021508B
:1009E00080409040E1F700C0000069E319C08338FF
:1009F00001F50E94D52080FD83C063E580916200EF
:100A0000909163000E9468210E94440E2FE789EABA
:100A100093E0215080409040E1F700C0000063E582
:100A200080916200909163000E946A21CF910C94A2
:100A3000440E8438C1F40E94D52082FD61C067E471
:100A400080916200909163000E9468210E94440E90
:100A50002FE789EA93E0215080409040E1F700C001
:100A6000000067E4DDCF8CEF8C0F813AD0F46C2F5F
:100A700080916200909163000E943221882349F0A6
:100A80006C2F80916200909163000E946A210E9405
:100A9000440E6C2F80916200909163000E94682147
:100AA000C5CF80E28C0F883048F4C77081E001C068
:100AB000880FCA95EAF70E94050EB8CFEBE5EC0F58
:100AC000E33040F4F0E0E554FF4F808190E0CF91B7
:100AD0000C94FA20E8E5EC0FE73150F4F0E0EE0F6B
:100AE000FF1FE357FF4F80819181CF910C9410211C
:100AF000CD3E30F08C2F0E948414CF910C9456156B
:100B0000CF910895882309F464C0823879F40E9453
:100B1000D52081FF5EC069E38091620090916300FF
:100B20000E9468210E94440E69E310C08338B1F42A
:100B30000E94D52080FF4DC063E5809162009091B6
:100B400063000E9468210E94440E63E58091620068
:100B5000909163000E946A210C94440E843879F4C9
:100B60000E94D52082FF35C067E480916200909199
:100B700063000E9468210E94440E67E4E7CF9CEF67
:100B8000980F913A10F4682FE1CF90E2980F9830C7
:100B900050F4877091E001C0990F8A95EAF7892F88
:100BA0000E940B0ED9CF9BE5980F933020F480E084
:100BB00090E00C94FA2098E5980F973120F480E0AB
:100BC00090E00C9410218D3E20F00E94DF140C94D4
:100BD000561508951F93CF93DF93182FEB010E94B2
:100BE000D804209741F087EB9BE00197F1F700C014
:100BF00000002197F6CF812FDF91CF911F910C94A8
:100C00008205893319F060E070E002C060E570E0B1
:100C10000C94EA05882321F00E94050E0C94440EE2
:100C20000895882321F00E940B0E0C94440E089521
:100C3000CF92DF92EF92FF920F931F93CF93DF93A8
:100C40007C01D62FC72FFC011281058102950F7000
:100C50000E94FB0D8823B9F01123A9F08C2F807F0F
:100C6000803421F080E28D0F883068F0809152024C
:100C700082FD09C082E00E94A40E0E94FB0D91E05B
:100C8000D82ED92601C0D12CCC2EC2948FE0C822F8
:100C90008C2D90E08C30910508F0CFC1FC01E65D11
:100CA000FF4F0C945B258C2F807FCF70882311F031
:100CB000C295C07F112399F0CC2309F4AAC180E228
:100CC0008D0F883010F0D11104C08C2F0E94050EBA
:100CD00003C08C2F0E94150E0E94440E9AC18D2FC6
:100CE0000E948205CC2309F4A8C180E28D0F8830D0
:100CF00038F1DD2329F18C2F0E941B0E24C08C2F8C
:100D0000807FCF70803211F0C295C07FDD2319F053
:100D1000D130A1F13DC08091520282FF17C0112352
:100D200049F0CC2329F08C2F0E94050E0E94440E1E
:100D300080E070C180E00E948205CC2309F47DC16F
:100D40008C2F0E940B0E0E94440E77C1112371F06C
:100D5000002341F0013031F40E94250E8C2B0E94BB
:100D60002D0E6BC10E94250E8C2B1DC0002319F087
:100D7000013009F462C10E943A0E25C0112321F00E
:100D8000063008F05AC10EC0053008F056C11BC02D
:100D9000112361F0002331F0F701858180FF39C113
:100DA0008F7085838C2F0E940A0647C1002359F05B
:100DB000D93309F03FC1FFEF0DEE12E0F1500040D2
:100DC0001040E1F735C18C2F0E94110636C18C2FDF
:100DD00086958695837019F0813061F02EC11123BC
:100DE00021F08D2F9C2F937002C080E090E00E9434
:100DF000FA202BC1112321F08D2F9C2F937002C05C
:100E000080E090E00E94102120C18D2F112319F065
:100E10000E94841402C00E94DF140E94561515C15E
:100E20008C2F837009F047C011110BC12D2F229513
:100E300026952770220F220F6D2F6F70862F90E05E
:100E4000A0E0B0E0022E04C0880F991FAA1FBB1FAC
:100E50000A94D2F7D4FF10C04FE050E060E070E099
:100E600004C0440F551F661F771F2A95D2F740957F
:100E700050956095709503C040E050E0BA01C6956A
:100E8000C695C3708A019B01082B192B2A2B3B2B7B
:100E9000C901B801C23049F058F4C13019F00E94BC
:100EA0001909CFC00E940709CCC00E942B09C9C0F4
:100EB0000E940509C6C0112319F08C2F817001C052
:100EC0008695882309F4BDC02D2F2295269527707D
:100ED000220F220F6D2F6F70862F90E0A0E0B0E000
:100EE000022E04C0880F991FAA1FBB1F0A94D2F7B5
:100EF000D4FF10C04FE050E060E070E004C0440F49
:100F0000551F661F771F2A95D2F74095509560951B
:100F1000709503C040E050E0BA01C695C695C37015
:100F20008A019B01082B192B2A2B3B2BC901B801E5
:100F3000C23049F058F4C13019F00E94DE0981C076
:100F40000E94CC097EC00E94F0097BC00E943F092C
:100F500078C0CF70112339F08C2F0E9465098D2F36
:100F60000E940A066EC08D2F0E9411068C2F0E94CF
:100F7000860967C0D23F21F128F4D03F41F0D13F2C
:100F8000C1F043C0D33F19F1D43F79F03EC01123E3
:100F900041F0053008F051C08C2F8F710E94AB09D1
:100FA0004CC0063008F049C0F7CF8091520282FF52
:100FB00018C0112339F08C2F8F710E9465093DC034
:100FC0001123C9F38C2F8F710E94860936C011231B
:100FD00029F08C2F8F710E9450092FC00E944B095D
:100FE0002CC0112349F0CF718C2F0E94650963E05A
:100FF0008C2F0E94890E21C081E00E94A40E023035
:10100000E0F082E00E94A40E18C0112331F000230A
:1010100091F28D2F0E94D80410C0002399F2D93389
:1010200049F41FEF2DEE32E0115020403040E1F73F
:1010300000C000008D2F0E94820588EF8C0D843047
:1010400020F40E94D5200E946D04DD20C9F00E948A
:10105000F70D80FD15C0F70112820E94F10D0E946C
:101060006509C7010E9461080E94F10DDF91CF91CF
:101070001F910F91FF90EF90DF90CF900C94860915
:10108000DF91CF911F910F91FF90EF90DF90CF9064
:1010900008950F931F93CF93DF93EC0168817981BB
:1010A0008A810E94A90A8C010E94020A0E94F30808
:1010B000B801CE010E941806DF91CF911F910F91C8
:1010C0000895CF93DF93EC01988189812B813C8136
:1010D000232B31F08F3F31F481E09F3F19F403C09F
:1010E00081E001C080E080FD1DC0CE010E940404AB
:1010F000811110C00E94FB0D8823A1F08A818823F2
:1011000089F08091520282FD0DC082E0DF91CF9183
:101110000C94A40ECE010E944908CE01DF91CF911C
:101120000C94E503DF91CF91089580E090E00E9458
:10113000FA2080E090E00E9410210E94220E0E947E
:10114000440E0E9487160C9456158091620090916F
:1011500063000E946C210C9495080E94120E0C945E
:10116000A50892959F70963079F010F4925001C0C6
:101170009A50923068F4803F69F018F4883E40F449
:1011800009C0843F29F406C0883E20F0813F11F059
:1011900080E0089581E00895FC01808191810E94A2
:1011A0009E0A0E94B1080895CF93DF9300D000D02B
:1011B0001F92CDB7DEB70F900F900F900F900F904A
:1011C000DF91CF910895CF93DF9300D000D000D06E
:1011D000CDB7DEB726960FB6F894DEBF0FBECDBFF3
:1011E000DF91CF910895089508950C94F4080C941C
:1011F000F5080E94F70860933501709336018093DB
:101200003701909338010C9495080C94F9080F93CA
:101210001F930091350110913601209137013091D3
:101220003801602B712B822B932B1F910F910C9403
:10123000F9080F931F930091350110913601209109
:1012400037013091380160237123822393231F914A
:101250000F910C94F9080F931F9300913501109191
:10126000360120913701309138016027712782279C
:1012700093271F910F910C94F9080C94F4080E9485
:101280003D09609331017093320180933301909353
:1012900034010C94950860E070E0CB010C943F0998
:1012A0000F931F9341E050E060E070E08A019B01E2
:1012B00004C0000F111F221F331F8A95D2F7C901E6
:1012C000B8011F910F910C943F090F931F9341E0B8
:1012D00050E060E070E004C0440F551F661F771FA8
:1012E0008A95D2F78091310190913201A09133011A
:1012F000B09134018A019B01082B192B2A2B3B2B1F
:10130000C901B8011F910F910C943F090F931F93CE
:1013100041E050E060E070E004C0440F551F661FDC
:10132000771F8A95D2F7409550956095709580917A
:10133000310190913201A0913301B09134018A01C1
:101340009B01082319232A233B23C901B8011F91BC
:101350000F910C943F090F931F9341E050E060E020
:1013600070E004C0440F551F661F771F8A95D2F79F
:101370008091310190913201A0913301B0913401FB
:101380008A019B01082719272A273B27C901B80191
:101390001F910F910C943F090F931F9300913101FE
:1013A000109132012091330130913401602B712B67
:1013B000822B932B1F910F910C943F090F931F9336
:1013C00000913101109132012091330130913401AB
:1013D00060237123822393231F910F910C943F0963
:1013E0000F931F930091310110913201209133012D
:1013F0003091340160277127822793271F910F9125
:101400000C943F090895292F220F920F990F890FED
:10141000E82FE695E695E695877051E001C0550FF7
:101420008A95EAF785E0E89FF0011124EE5DFE4F12
:1014300020E030E070E04081CB01022E02C09695A2
:1014400087950A94E2F78170819584278523842704
:1014500081932F5F3F4F2530310569F70895292F7C
:10146000220F920F990F890F682F669566956695E2
:10147000982F977085E0689FB001112440E050E0FC
:1014800080E0FB01E40FF51FEE5DFE4F208130E0B0
:10149000092E02C0369527950A94E2F7217033276A
:1014A000042E01C0220F0A94EAF7822B4F5F5F4F90
:1014B0004530510531F70895BF92CF92DF92EF92F8
:1014C000FF920F931F93CF93DF938C01C090310154
:1014D000D0903201E0903301F090340180913501D9
:1014E00090913601A0913701B0913801C82AD92ACC
:1014F000EA2AFB2ACFE1D0E0D701C6010C2E04C0B6
:10150000B695A795979587950A94D2F780FD04C064
:10151000219790F7B12C07C0BC2EB8018C2F0E94E8
:1015200094110197A9F38B2DDF91CF911F910F910A
:10153000FF90EF90DF90CF90BF900895CF93DF930F
:10154000EC010E945C0ABE010E949411DF91CF91D0
:1015500008951F93CF93DF93EB019091210199237D
:1015600021F0CB010E949E0A13C0882349F0CB01D1
:101570000E945C0A182F682FCE010E94030A04C043
:10158000CB010E942F0A182FBE01812F0E949411B7
:10159000DF91CF911F9108951F93CF93DF93C09157
:1015A000390116E080913A01C81799F0D0E01C9FEC
:1015B000F0011D9FF00D1124E55CFE4F408151812B
:1015C00062817381848195810E94E3082196C770AE
:1015D000E9CFDF91CF911F91089540916B01509118
:1015E0006C0160916D0170916E0180916F0190911D
:1015F00070010C94E308EF92FF920F931F93CF9327
:10160000DF938091700182958F7009F065C08091A1
:101610006D01882309F460C080913901F0903A018E
:1016200010916B0100916C0160916E0170916F01DE
:1016300091E01F3F09F090E0C0916000D0916100FF
:10164000292F96E0E92E8F1509F446C06115710522
:1016500021F00F3F21F030E003C031E001C0322F14
:1016600090E030FD36C0E89EF001E99EF00D1124B7
:10167000DF01A55CBE4F11963C911197301329C034
:101680003C91311326C012963C911297311121C022
:1016900013964D915C911497461B570B4C175D07A1
:1016A000C0F4809170018F70806180937001E05C64
:1016B000FE4F80818F70806180838BE691E00E9475
:1016C0006108DF91CF911F910F91FF90EF900C94E3
:1016D000CC0A01968770B7CFDF91CF911F910F9100
:1016E000FF90EF9008959F92AF92BF92CF92DF92BA
:1016F000EF92FF920F931F93CF93DF93CDB7DEB797
:1017000061970FB6F894DEBF0FBECDBF8C0185E0A8
:10171000F801DE011D9601900D928A95E1F7D8013E
:101720001296EC9090916B01E0916C0120916E010A
:1017300030916F012115310531F0EF3F31F481E037
:101740009F3F19F403C081E001C080E0B82FB17061
:101750009B2E80FD47C1D8014C9111965C91119749
:101760001396AD90BC9014978BE6C82E81E0D82ECE
:10177000F0906D01B501621B730B209160003091F8
:101780006100FF2009F4D9C08091700162177307CE
:1017900008F095C0282F207F09F052C05E1313C0B7
:1017A000491311C0FE2CE1100EC08F708061809330
:1017B00070010E94ED0AC6010E94610880917001CB
:1017C000F80185834DC1AB2831F05F3F31F481E0F2
:1017D0004F3F19F403C081E001C080E080FD03C0E9
:1017E00081E08E2502C080E090E0F82FF170FF2E9E
:1017F00080FF1CC08091390120913A0136E08217A8
:1018000009F40BC190E0389FF001399FF00D1124CD
:10181000E55CFE4F6181561306C06081461303C02C
:101820006281E61203C001968770E9CFFE2CEE209C
:1018300009F416C18091700181608093700154C0D9
:101840005E1306C0491304C0E11002C0F80199C03C
:10185000C8010E94CC08882361F1EE2051F120914B
:101860007001822F82958F7090E0029774F08091C2
:101870006B0190916C0198878F831986BB86AA862D
:101880002C87CE0107960E94610886E0F801ABE63E
:10189000B1E001900D928A95E1F70E94FB0A0E9447
:1018A000ED0A0AC05E1711F1C8010E94CC0881112F
:1018B0002CC0C8010E946108FF24F394D1C0282FD6
:1018C000207F81F77A2DB98AA88A6E2D89890E9496
:1018D000D4088BE691E00E94610886E0D6011D9253
:1018E0008A95E9F70E94ED0AF12CBAC04913DCCFC2
:1018F000E110DACFF8018583C8010E94610886E013
:10190000D6011D928A95E9F7ABC0EE2091F22091A5
:101910007001822F82958F7090E002970CF4B5CF02
:1019200080916B0190916C019A8389831B82BD82A7
:10193000AC822E83CE010196A6CF6217730708F002
:1019400044C0FE2CEE2009F4B4CF5E1330C049131E
:101950002EC02091700120FD21C0822F82958F70B2
:10196000482F50E041155105C9F0F80125834F304B
:10197000510541F08F5F982F9295907F822F8F7045
:10198000892B8583C8010E94610886E0F801ABE6D7
:10199000B1E001900D928A95E1F73CC086E0F80134
:1019A000ABE6B1E001900D928A95E1F759C0C8010C
:1019B0000E94CC08811169CF809170018160809371
:1019C0007001C8010E9461084BC07A2DB98AA88AAB
:1019D0006E2D89890E94D40886E0D6011D928A95D1
:1019E000E9F718C0EE2009F464CFC8010E94CC08C2
:1019F000F82E882309F45DCF86E0F801ABE6B1E06C
:101A000001900D928A95E1F78BE691E00E94D20455
:101A10000E94FB0A0E94ED0A23C04D875E878D85D8
:101A20009E850E949E0A292F22952F70223028F42D
:101A30009F7039F0811105C00BC0243028F49F70CD
:101A400049F4805E883020F0C8010E9461089F2C14
:101A5000F92C06C0D80115969C91907F91F7F8CF8C
:101A60008F2D61960FB6F894DEBF0FBECDBFDF910C
:101A7000CF911F910F91FF90EF90DF90CF90BF908B
:101A8000AF909F9008951F93CF93DF93CDB7DEB7AC
:101A90002C970FB6F894DEBF0FBECDBF4F8358878B
:101AA00069877A878B879C87CE0107960E94730B84
:101AB0008823D1F09F8188852A853B85232B31F0AF
:101AC0008F3F31F481E09F3F19F403C081E001C0F2
:101AD00080E080FD47C04F81588569857A858B8578
:101AE0009C850E94E3083EC086E0FE013796DE0139
:101AF000119601900D928A95E1F7FF81E8856A853C
:101B00007B856115710531F0EF3F31F481E0FF3FD6
:101B100019F403C081E001C080E080FD23C0209162
:101B20003A0130E0C9010196877099274091390147
:101B300050E084179507F1F1F983EA837D836C8384
:101B400096E0929FD001939FB00D1124A55CBE4FEB
:101B5000FE01319601900D929A95E1F780933A013A
:101B60000E94CC0A16E08091390190913A018917C0
:101B700071F1189FC0011124855C9E4F0E94730B68
:101B8000882329F1E09139011E9FF0011124E55CC1
:101B9000FE4F4081518162817381848195810E94D1
:101BA000E3088091390190E001968770992780932E
:101BB0003901D9CF0E94AD0810923A011092390133
:101BC000EBE6F1E086E0DF011D928A95E9F72C96BD
:101BD0000FB6F894DEBF0FBECDBFDF91CF911F913E
:101BE00008958091790185958595859508958091D1
:101BF00079018770089590917901977081E009F4D7
:101C000080E0089580918401089590918401892B4A
:101C10008093840108958095909184018923809315
:101C20008401089510928401089590918301892B75
:101C300080938301089580959091830189238093F7
:101C40008301089510928301089580917A01089587
:101C500008950C94280E0C94290E9091520292FD36
:101C600008C090917A01981721F080937A010C9422
:101C70002B0E089580917A01882329F010927A0121
:101C800080E00C942B0E0895CF93DF93E0916200D7
:101C9000F0916300809184018083E0916200F09173
:101CA0006300908180918301892B808380917A01E8
:101CB000882381F0E0916200F09163009081892B8C
:101CC000808380916200909163000E94262181119F
:101CD0000E943A0EC0916200D091630048E050E04B
:101CE00061E771E0CE010E94AB25892B69F088E0A5
:101CF000FE01A1E7B1E001900D928A95E1F7CE01D6
:101D0000DF91CF910C94E120DF91CF9108950C9455
:101D1000280E9091520292FD10C098E0899F900188
:101D20001124262B209379010E9465098091790165
:101D30008595859585950C94870E0C946509109270
:101D4000790180E00C94870E20917901809582239F
:101D500080937901982F977099F430E0482F082EDE
:101D6000000C550B2417350759F09091520292FD43
:101D700007C08595859585950E9486090C949F0ED0
:101D800008959091520292FB222720F9281769F0BA
:101D900080FB92F9909352028091510290915202ED
:101DA0000E940F0F82E00C94A40E089580915202BD
:101DB00082FB882780F991E089270C94C10E81E08D
:101DC0000C94C10E80E00C94C10E6FEF7FEF80E0A9
:101DD00090E00C94E92580E090E00E94C62521E087
:101DE000893E9E4F09F020E0822F089582E090E026
:101DF0000C94B82583E090E00C94B825CF9384E050
:101E000090E00E94B825C82F82E290E00E94B82599
:101E10002C2F30E0A901582BCA01CF910895CF9300
:101E2000C92F682F84E090E00E94CC256C2F82E2BD
:101E300090E0CF910C94CC25AB01BC018FE090E0F9
:101E40000C94DD25AB01BC0183E190E00C94DD2511
:101E500060E070E0CB010C94220F60E070E0CB01F9
:101E60000E941C0F0C94280F69EE7EEF80E090E03A
:101E70000E94E92560E082E090E00E94CC2560E0CD
:101E800083E090E00E94CC2510923501109236013B
:101E9000109237011092380160E084E090E00E94D7
:101EA000CC2560E082E290E00E94CC2560E085E0F5
:101EB00090E00E94CC2560E086E090E00E94CC2576
:101EC0006FEF87E090E00E94CC2540E050E0BA013F
:101ED00088E090E00E94DD2560E08DE090E00E94C7
:101EE000CC2540E050E0BA0188E190E00E94DD2579
:101EF00060E087E190E00E94CC2540E050E0BA012C
:101F00008CE190E00E94DD2560E070E080E290E0EE
:101F10000E94E92540E050E0BA0188E190E00E948B
:101F2000DD250C942D0F0C94340F682F8EE090E07B
:101F30000C94CC250E94B02160938D0170938E018A
:101F400080938F01909390016093890170938A012F
:101F500080938B0190938C01089584B7806884BF2F
:101F600084B7806884BF089581E008950C94B40F0D
:101F700008950C94B80F0C94B80F0C94BB0F0C94EC
:101F8000B80F0C94BF0F0C94B80F0E94AD0F80E7F0
:101F900092E10E94CB200E94C30F0C94C10F0E94BB
:101FA000B90F0C94B80F0E948A120C946C040E9412
:101FB0009D210E9466130E94D30F0E94E61B0C9481
:101FC000BD0F8F929F92AF92BF92CF92DF92EF920E
:101FD000FF920F931F93CF93DF93CDB7DEB72A976E
:101FE0000FB6F894DEBF0FBECDBF0E947B13982EB4
:101FF00081110E949A0F85E8A82E81E0B82E00E09A
:1020000010E0802E802F0E94AE12D82EF501C190D4
:102010005F01C826B1F40F5F1F4F0430110589F727
:102020008FEF89838A831B820E94A4218160782F8D
:102030009D838C8349815A816B818D810E948804A4
:102040002FC08091910181FD0E94B412E12CFF24E8
:10205000F3948C2D8F21F1F00E94B60F882399F014
:10206000EE828F82DF2081E009F480E088870E9481
:10207000A4218160782F9A8789874E815F81688546
:102080008A850E948804F801EB57FE4F8081F8266C
:10209000F08206C0E394FF0CF6E0EF12DACFBBCF7C
:1020A00081E0911001C080E02A960FB6F894DEBF5F
:1020B0000FBECDBFDF91CF911F910F91FF90EF9099
:1020C000DF90CF90BF90AF909F908F9008950E9427
:1020D000E10F0E94191C0E9474150C947D04CF938B
:1020E000DF930E949911EC01811521E5920708F018
:1020F00045C0811530E5930708F094C0883E9105EE
:1021000028F5803E910508F0F8C0883A910570F4F2
:10211000853A910508F07CC08130910509F475C0BD
:1021200008F4E8C0049708F0E8C0E4C08F3B9105CC
:1021300008F0E0C0C85AD0E0CC0FDD1FC254DF4F1A
:102140000990D881C02DCE019464D8C0811540E299
:10215000940758F4811551E0950708F0CEC08D3EE4
:10216000910508F4C7C09065C9C0C11580E4D807BF
:1021700008F4C0C0DF70CE01906AC0C0811525E5AB
:102180009207A8F4811534E5930708F095C08115EE
:1021900043E5940708F07BC0811552E5950708F0E8
:1021A00061C0D82FCC27CE01816F906AA7C0C1151E
:1021B00089E5D807A0F4C11528E5D20708F082C048
:1021C000C11536E5D30708F095C08C2F0E942D125B
:1021D0008F7190E0D82FCC27CE0190628FC0C115AF
:1021E0004AE5D40708F474C0CE0190568115904298
:1021F00008F080C08D2F8F710E942D12DD27D062D4
:102200008F71AE01582BCA0179C081E090E076C091
:10221000C55AD0E0C451DF4F8881C82FD0E0CE012D
:1022200090646CC074E0969587957A95E1F7282FB5
:1022300023703C2F337081E090E002C0880F991F1B
:102240003A95E2F79C68AC01522B9A019C2F9F7043
:102250009695969550E2959FE0011124C9018C2B2B
:102260009D2B4CC08370992721E030E002C0220FE3
:10227000331F8A95E2F79C2F9695969580E2989F5A
:10228000E0011124C22BD32BCE019C6837C0837090
:10229000992721E030E002C0220F331F8A95E2F730
:1022A0009C2F9695969540E2949FE0011124C22BB5
:1022B000D32BCE019A6822C0D82FCC27CE01846FB1
:1022C000906A1CC0DC2FCC27CE01806F906A16C0AC
:1022D0008C2F8F700E942D1294E0D695C7959A95F9
:1022E000E1F7CF70D0E0DC2FCC27D0699E01282BFE
:1022F000C90104C080E090E001C0CE01DF91CF9120
:10230000089528E1829FC0011124FC0126E0729FFC
:10231000E00DF11D1124E60FF11DEE0FFF1FE45932
:10232000FF4F8591949108950E9481110E946F1032
:1023300008958238910569F1B0F48133910509F46B
:102340006DC048F48932910509F463C08A32910561
:1023500009F469C008958533910509F455C089339E
:102360009105B9F00895833E910569F138F4803EF6
:102370009105B1F0823E910509F10895863E9105DF
:10238000A9F1873E9105B9F1843E910509F064C039
:1023900023C02091510220FD4FC021FD4DC0089562
:1023A0008091510280FD44C08091520280FF44C060
:1023B0008091510284FD42C083EE4DC08091510254
:1023C00082FF38C0F5CF8091510282FD33C08091E9
:1023D000520280FD31C0ECCF8091520281FF32C0A9
:1023E0008091510284FD2AC087EE35C08091510250
:1023F00083FF26C0F5CF8091510283FD21C08091DB
:10240000520281FD1FC0ECCF8091510285FD1CC09E
:102410001DC08091510285FD19C016C080915102E6
:1024200086FD16C017C08091510286FD13C010C0F2
:1024300089E311C082EE0FC080EE0DC080E00BC0BA
:1024400086EE09C084EE07C089E205C085E303C0BB
:102450008AE201C081E390E008959091510292FFD9
:102460000DC0282F2871283019F4877F846006C09A
:10247000282F2471243011F48B7F886093FF0DC0C6
:10248000282F2871283119F4877E846106C0282FEF
:102490002471243111F48B7E88612091520220FF37
:1024A0000DC0382F3871383019F4877F816006C02D
:1024B000382F3171313011F48E7F886021FF0DC0CB
:1024C000282F2871283119F4877E816106C0282FB2
:1024D0002171213111F48E7E886194FD877E0895EB
:1024E00080E008950C94E50E0E947B138FE295E73F
:1024F0000197F1F700C000000E947B1380E00E946A
:10250000AE1280FF04C00E9472120C94F121089553
:102510000C9474120E94EB0E811102C00E94930F62
:102520000E94F60E809391010E94FE0E909352023B
:10253000809351020E9488120E94FA0E682F70E068
:1025400080E090E00E9405096091310170913201B4
:1025500080913301909134010C943D09E82FF0E013
:10256000E95AFD4F80810895089588E78A95F1F72B
:10257000089500C008950C94B51208950C94BD12EE
:102580000C94BE120C94BD120C94C212F894E82F55
:10259000E295EF70F0E031A9282F2F7081E090E0F4
:1025A00001C0880F2A95EAF7982F9095932391AB55
:1025B00092A9892B82AB789408950F931F93CF93A0
:1025C000DF93CFEED0E089918F3F11F00E94C612C9
:1025D00080E0C53FD807B9F7C5EFD0E009EF10E0BC
:1025E00089918F3F11F00E94C6120C171D07C1F789
:1025F000DF91CF911F910F910895EF92FF920F936A
:102600001F93CF93DF93C62FD0E0C151DF4F2881B6
:102610002F3F09F454C0042F162F7C01F894E22FA9
:10262000E295EF70F0E081A9422F4F7021E030E099
:1026300001C0220F4A95EAF7822B81AB82A920952F
:10264000282322AB78940E94B91265EF70E0F7015D
:10265000A7014C5F5F4FF12C302F3095DB012D919E
:10266000BD012F3FB1F0822F82958F7090E0DC0189
:10267000D0968C9190E02F7002C0959587952A9501
:10268000E2F780FD06C08081802B8083FF24F394D5
:1026900003C08081832380833196E417F507F1F628
:1026A00088818F3F11F00E94C6126F2D812FDF911C
:1026B000CF911F910F91FF90EF900C94BB12DF917F
:1026C000CF911F910F91FF90EF9008950E94DD121E
:1026D00084E0E7E5F2E0DF01982F1D929A95E9F793
:1026E000E3E5F2E0DF011D928A95E9F784E00E94BC
:1026F000C2130C94F0030F931F93CF93DF9300D07A
:1027000000D0CDB7DEB719821A821B821C8210E07E
:1027100001E0402F612FCE0101960E94FD121F5F44
:10272000000F1630B1F744E050E0BE016F5F7F4FFD
:1027300083E592E00E94AB2511E0009709F410E0D8
:10274000892B61F089819A81AB81BC81809353028E
:1027500090935402A0935502B0935602212F44E067
:1027600067E572E083E592E00E94C3130E94F203E2
:10277000812F0F900F900F900F90DF91CF911F91AD
:102780000F9108950895FF920F931F93CF93DF93B6
:102790008C01F62ED72FC42F222349F081E080939D
:1027A00094010E94A42190939301809392018091BF
:1027B00094018823C1F080919201909193010E942D
:1027C000BC21059780F0EF2DFD2FD8014C2F50E054
:1027D000CD01801B910B841795071CF48D9181937B
:1027E000F7CF10929401DF91CF911F910F91FF903D
:1027F00008950E9406220E94D70F0C9417220E946F
:1028000092210E94FF210E94C50F0E94F9130E948D
:1028100025220E94CF0FFBCF80919B0180FF06C035
:102820006091690070E0660F771F26C081FF04C0C9
:102830006091690084E005C082FF07C06091690073
:1028400088E0689FB001112417C090919A019923E4
:10285000D1F060916800961788F72091690088E0B0
:10286000289F90011124929FA001939F500D112445
:1028700070E0CA010E9425256038710540F4611599
:10288000710519F406C068E070E0862F08958FE79F
:10289000089581E0089580919B0180FF08C06091B8
:1028A000650070E0759567957595679521C081FF06
:1028B00006C06091650070E07595679519C082FF4C
:1028C00004C06091650070E010C090919901992357
:1028D00099F0609164009617A0F780916500899F38
:1028E000C001112470E00E9425256038710540F474
:1028F0006115710519F406C061E070E0862F089536
:102900008FE7089581E008958D3E21F40E940C1414
:10291000819504C08E3E29F40E940C1480939F017F
:1029200008958F3E21F40E940C14819504C0803FCD
:1029300029F40E940C1480939E010895893F19F494
:102940000E944B1405C08A3F31F40E944B148195BC
:102950008093A00108958B3F21F40E944B14819530
:1029600004C08C3F29F40E944B148093A101089568
:102970009FE0980F983078F421E030E0A90102C080
:10298000440F551F9A95E2F7CA0190919D01892B3A
:1029900080939D0108958D3F21F480919B0181607A
:1029A0000BC08E3F21F480919B01826005C08F3F58
:1029B00029F480919B01846080939B0108958D3E52
:1029C00039F490919F0197FF35C010929F0159C033
:1029D0008E3E29F490919F011916BCF32BC0909163
:1029E0009E018F3E29F497FF25C010929E0149C099
:1029F000803F19F41916CCF31DC09091A001893FB6
:102A000029F41916BCF41092A0013BC08A3F19F4B6
:102A100097FF10C0F8CF8B3F39F49091A10197FF39
:102A200009C01092A1012DC08C3F21F49091A10109
:102A30001916BCF39FE0980F983080F421E030E045
:102A4000A90102C0440F551F9A95E2F7CA0180956B
:102A500090919D01892380939D0113C08D3F21F4A6
:102A600080919B018E7F0BC08E3F21F480919B0152
:102A70008D7F05C08F3F29F480919B018B7F8093D0
:102A80009B0180919E01811106C080919F0181115F
:102A900002C010929A018091A001811106C080911C
:102AA000A101811102C01092990108950E94A421F0
:102AB00020919E01211104C020919F01222321F029
:102AC00090939801809397012091A001211104C057
:102AD0002091A101222321F09093960180939501EA
:102AE0008CE991E00C94EC20EF92FF920F931F93EE
:102AF000CF93DF9300D000D000D0CDB7DEB786E013
:102B0000ECE9F1E0DE01119601900D928A95E1F772
:102B1000E0909E01F0909F010091A0011091A10111
:102B200010929E0110929F011092A0011092A1019B
:102B3000E11003C0FF2009F45DC0809197019091DE
:102B400098010E94BC21AC0190919A01992339F01F
:102B500020916A0030E02417350758F04BC02091CF
:102B60006B008AE0289F900111242417350718F084
:102B700041C09F3F19F09F5F90939A01EE2061F052
:102B80000E940C141E1414F09FEF01C091E0989F56
:102B9000902D112490939E01FF2061F00E940C144F
:102BA0001F1414F09FEF01C091E0989F902D112405
:102BB00090939F0130919E013323E1F020919F017A
:102BC0002223C1F045EB3403C0011124992319F0ED
:102BD00090939E0103C081E080939E0135EB230317
:102BE000C0011124992319F090939F0103C081E043
:102BF00080939F01011103C0112309F45DC08091EE
:102C00009501909196010E94BC21AC01909199018F
:102C1000992339F02091660030E02417350758F0E9
:102C20004BC0209167008AE0289F9001112424174F
:102C3000350718F041C09F3F19F09F5F90939901AD
:102C4000002361F00E944B14101614F09FEF01C096
:102C500091E0989F902D11249093A001112361F091
:102C60000E944B14111614F09FEF01C091E0989F41
:102C7000902D11249093A1013091A0013323E1F014
:102C80002091A1012223C1F045EB3403C00111249E
:102C9000992319F09093A00103C081E08093A001D3
:102CA00035EB2303C0011124992319F09093A1015E
:102CB00003C081E08093A10180919E0181110BC02E
:102CC00080919F01811107C08091A001811103C0F3
:102CD0008091A10181110E945615EB82FC820D8327
:102CE0001E8386E0FE013196ACE9B1E001900D92C1
:102CF0008A95E1F726960FB6F894DEBF0FBECDBFDA
:102D0000DF91CF911F910F91FF90EF900895ECE923
:102D1000F1E086E0DF011D928A95E9F710929A01B1
:102D20001092990110929B010895EF92FF920F93D8
:102D30001F93CF93DF938B01682F11110AC0442397
:102D400029F0E82FF0E0ED51FE4F6491762F862FA9
:102D500075C0212F30E0E82FF0E0442321F0ED5141
:102D6000FE4FE491F0E046E0049FC0011124CFEF54
:102D7000D0E0BE010E9411254BEA4603C001479FE7
:102D8000900D1124800F911D800F911D982F990F88
:102D9000890FAE01421B530B4E9FD0014F9FB00DC8
:102DA0005E9FB00D11249B2F189FA0011124452F69
:102DB00055278E01041B150B0E9FA0010F9F500D70
:102DC0001E9F500D11247E01E81AF108E29E800139
:102DD000E39E100DF29E100D1124212F3327C21BEC
:102DE000D30BCE9F9001CF9F300DDE9F300D11246D
:102DF00062307105A9F048F46115710569F0613020
:102E00007105C9F48B2F752F0DC06430710581F0E9
:102E100058F06630710579F47E2F8B2F932F0DC0FB
:102E2000832F7B2F9E2F09C08E2F7B2F952F05C0C0
:102E30008E2F732F02C07E2F852F692FDF91CF91A8
:102E40001F910F91FF90EF90089541E00E94951619
:102E5000089508950E9425170895CF93DF93762F44
:102E6000E901682F842F0E942A17798368838A8357
:102E7000DF91CF91089580915B02282F269530E055
:102E80002115310519F48170826005C025323105A4
:102E900024F08170886480935B02089588E090E05C
:102EA0000C94C025CF92DF92EF92FF926B017C01D0
:102EB0000E943B17B701A60188E090E0FF90EF90D9
:102EC000DF90CF900C94DD25EBE5F2E083E080838A
:102ED00011828FEF8283838314826081718182816A
:102EE00093810C94521780915B0280FF02C08695FB
:102EF000089580E0089590915F02933018F49F5FE9
:102F000090935F02882351F060915B0270915C02A4
:102F100080915D0290915E020C945217089581E0B9
:102F20000C947B1790915F02992319F09150909324
:102F30005F02882351F060915B0270915C02809186
:102F40005D0290915E020C945217089581E00C94FA
:102F5000921770E00C94961D6091700080915B0256
:102F600080FF0AC080916F0023E0829FC00111247E
:102F7000805A9D4F0C94A917809171009091720016
:102F8000891780F7E82FF0E09F01220F331FE20F2F
:102F9000F31FE05AFD4F1182108212828F5FF0CF33
:102FA00090915B0290FF16C0909171002091720089
:102FB000921770F4E92FF0E0DF01AA0FBB1FEA0FB0
:102FC000FB1FE05AFD4F8183608342839F5FF0CFF8
:102FD0000C94AC170895CF93DF9300D01F92CDB718
:102FE000DEB790915B0290FF0AC09E012F5F3F4FBA
:102FF0000E942D174B8169818A810E94D0170F9002
:103000000F900F90DF91CF910895CF93DF93EC0154
:10301000EC81F0E0E252FF4F4491EBE5F2E0628197
:1030200081810E94EB178C818F5F8C83DF91CF9120
:103030000895CF93DF93EC01EBE5F2E043816281E9
:103040008C810E94EB178C818F5F8C83DF91CF91F5
:1030500008950F931F93CF93DF9300D01F92CDB7A6
:10306000DEB78C018091A20181110AC09E012F5F01
:103070003F4F4FEF6FEF0E942D178A818093A2017F
:10308000F8018481813051F028F0823061F4409160
:10309000A2010AC08091A20140E007C06091A20194
:1030A00040E080E003C040E080E060E00E94D01794
:1030B000F801848190E0019663E070E00E9425258C
:1030C00084830F900F900F90DF91CF911F910F91FC
:1030D0000895AF92BF92CF92DF92EF92FF920F933B
:1030E0001F93CF93DF9300D01F92CDB7DEB7182F79
:1030F000F62E042FE22E90915B0290FF6DC0E92F17
:10310000E695AE2FB0E0A750BF4F8C918093AC01F5
:103110009E7F923061F49E012F5F3F4F812F0E946E
:103120002D174B8169818A810E94D01743C082305C
:1031300019F400915E023EC0863019F410915C02D1
:1031400039C08930D9F38931A9F5E9518E2F8170C1
:10315000D82EE695F0E0E252FE4FA590B490C12C37
:10316000BB2460917300C61618F52C2D30E0A29E8A
:10317000C001A39E900DB29E900D112470E00E949C
:103180001125812FD11002C0860F01C0861B90919E
:103190007100290F311DA901440F551F240F351F40
:1031A000205A3D4F402F6F2D0E942D17C394D9CF29
:1031B0000E94AC1710935C02F0925D0200935E02D5
:1031C000EE2051F060915B0270915C0280915D0293
:1031D00090915E020E9452170F900F900F90DF9116
:1031E000CF911F910F91FF90EF90DF90CF90BF9004
:1031F000AF900895EBE5F2E09181282F4381628141
:1032000088E0890F0C94691881E00C94FA18EBE5BA
:10321000F2E09181282F4381628188EF890F0C941D
:10322000691881E00C940719EBE5F2E0628128E06F
:10323000620F08F46FEF282F438181810C94691885
:1032400081E00C941419EBE5F2E0628128E0621B46
:1032500008F460E0282F438181810C94691881E093
:103260000C942319EBE5F2E0438128E0420F08F4C7
:103270004FEF282F628181810C94691881E00C94B2
:103280003219EBE5F2E0438128E0421B08F440E00C
:10329000282F628181810C94691881E00C94411976
:1032A00020E00C946918FF920F931F93CF93DF9344
:1032B000EC01F12C0FEF10E060917300F616F0F4C2
:1032C000809171002F2D30E0280F311DC901880F2A
:1032D000991F280F391F205A3D4F70E0C8010E94E6
:1032E0002525962F8C8140915E0260915D02F99EAA
:1032F000800D11240E942D17F394DECF0E94AC178D
:103300009A818C8190FF02C08F5F01C081508C83B5
:10331000DF91CF911F910F91FF900895AF92BF92CF
:10332000CF92DF92EF92FF920F931F93CF93DF9391
:10333000FC01828180FF02C00FEF01C001E010E0BC
:1033400047E0A42E80917300181708F043C08091C5
:103350007100C12ED12CE601C80FD11DCE01880FFE
:10336000991FC80FD91FC05ADD4F198218821A82BF
:1033700034E0E32EF12CB12C8091A4018B0D883028
:103380002CF06A2D0E940325892F05C087FF03C0FA
:1033900090917300890F082E000C990BC816D9065E
:1033A00091F480915E028E9DA0018F9D500D11249D
:1033B00055954795559547959E0160915D02809181
:1033C0005C020E942D17B00EF1E0EF1AF108A1F691
:1033D0001F5FB8CF0E94AC178091A401013031F477
:1033E000811102C080917300815007C090E0019666
:1033F0006091730070E00E9425258093A401DF9105
:10340000CF911F910F91FF90EF90DF90CF90BF90E1
:10341000AF900895CF9380917100909172008917B9
:1034200070F4E82FF0E09F01220F331FE20FF31F2B
:10343000E05AFD4F1182108212828F5FF0CFC0E000
:1034400060917300C617C0F5EC2FF0E070E0CF017B
:103450000E94252520917100820F2091A301022E48
:10346000000C330B90E0E217F307CCF020916E00D4
:10347000022E000C330B2E173F078CF09C01220FFD
:10348000331F820F931F9C01205A3D4F40915E02D3
:1034900060915D0280915C020E942D170BC0FC01BF
:1034A000EE0FFF1F8E0F9F1FFC01E05AFD4F118290
:1034B00010821282CF5FC4CF0E94AC1720916D00A2
:1034C0008091A301820F8093A30190916E00920FCF
:1034D00090936E0019165CF4082E000C990B409125
:1034E000730050E041505109841795071CF0219555
:1034F00020936D00CF9108958F929F92AF92BF92CB
:10350000CF92DF92EF92FF920F931F93CF93DF93AF
:103510008C01FC014481C42FD0E09E01DE010E9499
:1035200069259B01AC010E947F256B017C01E0E2D3
:10353000F0E0EC1BFD0BA5E5B0E09B01AC010E94A7
:103540007F254B015C019F01DF010E9461259B01EA
:10355000AC010E948A259B01AC012C0D3D1D4E1D26
:103560005F1DC501B4010E943925C22FD22F2A3216
:1035700028F4F3E02F9F900111240DC025E530E0E1
:103580002C1B3109C901880F991F280F391F37FFDC
:1035900002C02F5F3F4F35952795C22FC095F12C64
:1035A00085E5E82EED1A80917300F816C8F4F1FC59
:1035B00002C08E2D01C08D2F909171002F2D30E013
:1035C000290F311DA901440F551F240F351F205A03
:1035D0003D4F4C2F60915D020E942D17F394E3CF75
:1035E0000E94AC17F8018481811102C091E003C0F0
:1035F000803219F49FEF90936C0090916C00890FCA
:10360000F8018483DF91CF911F910F91FF90EF908C
:10361000DF90CF90BF90AF909F908F9008950F93C1
:103620001F93CF93DF93EC0100E010E080917300D3
:10363000282F30E00217130724F5909171009801AC
:10364000290F311DA901440F551F240F351F205A82
:103650003D4F869590E04C81081719071CF44423D0
:1036600031F002C0411103C040915E0201C040E050
:1036700060915D0280915C020E942D170F5F1F4FC9
:10368000D5CF0E94AC178C8190E00196817099276C
:103690008C83DF91CF911F910F910895EBE5F2E0BC
:1036A00080818E7F808360817181828193810E947D
:1036B00052171092AD012FEB84ED91E02150804024
:1036C0009040E1F700C000000C94AC1760915B02E1
:1036D000669570E04BE050E084E790E00E949E2504
:1036E000892B19F481E08093AD010E94A42190936D
:1036F000A6018093A501089590915B0290FF35C0CB
:103700009170811102C0926006C0853210F09864F9
:1037100002C0880F982B90935B02662351F0609152
:103720005B0270915C0280915D0290915E020E944A
:10373000521760915B02669570E04BE050E084E7C1
:1037400090E00E949E25892B19F01092AD0102C0D5
:103750000E94661B81E08093A80140915E02609107
:103760005D0280915C020C9450190895682F90912D
:103770005B02969581E0890F853208F081E00C9418
:103780007C1B81E00C94B61B682F90915B02969590
:103790008FEF890F09F484E20C947C1B81E00C9478
:1037A000C41B61E00C947C1BEBE5F2E0808181603E
:1037B000808386950C94D11B80915B0280FD0C94D4
:1037C0004E1B0C94D41B60E00C947C1B8091AB01CD
:1037D00081112EC00E94EB0E811104C00E94930F34
:1037E0000E9464170E944E1760935B0270935C0204
:1037F00080935D0290935E026E7F61F40E94641775
:103800000E944E1760935B0270935C0280935D028E
:1038100090935E020E943B171092AD0180915B0273
:1038200080FF03C086950E94E31B81E08093AB017B
:1038300008950F931F93CF93DF938091AD01882359
:1038400009F485C08091AC01E0915B02E695E81B2C
:10385000E093A701823049F4F0E0E652FF4FE49193
:10386000CE2FD0E005E018E149C0863049F4F0E001
:10387000E952FF4FE491CE2FD0E009E118E13EC0BC
:10388000893051F4E695F0E0EC52FF4FE491CE2FF1
:10389000D0E003E519E132C08F3051F4E695F0E055
:1038A000EF52FF4FE491CE2FD0E00EE819E126C091
:1038B000853149F4F0E0E253FF4FE491CE2FD0E0A0
:1038C0000AE01AE11BC0883181F0833239F4ECEC54
:1038D000F0E0C591D49109E218E110C0843251F4AE
:1038E000C4EFD1E00FE01BE109C0C8E2D0E00CE773
:1038F0001AE104C0C0EDD7E009E217E18091A80108
:10390000882361F01092A8010E94A4219093A6013F
:103910008093A5011092AA011092A9010E94A421EE
:10392000E091A501F091A6018E1B9F0B8F3F9F4751
:1039300070F4EC0FFD1FF093A601E093A50185EA5A
:1039400091E0F801DF91CF911F910F910994DF91E0
:10395000CF911F910F910895882311F0FA0101C0B2
:10396000FB010994CF93DF93C82FD62F0E947317C2
:103970008C1740F00E9473178D1720F4DF91CF91C0
:103980000C94C11B8C2FDF91CF910C94D11B1F93F2
:10399000CF93DF93FB0112811111C3C0EC010E9490
:1039A000020E8272CD3CFCE5DF0709F49AC0A8F54F
:1039B000C73CECE5DE0709F476C0A8F4C43C9CE5FE
:1039C000D90709F45FC028F4C33CDC4509F457C0AB
:1039D00054C0C53C9CE5D90709F459C0C63CDC4538
:1039E00009F45CC04AC0CA3CFCE5DF0709F46AC0C0
:1039F00050F4C83CECE5DE0709F45AC0C93CDC458C
:103A000009F45BC03AC0CB3C9CE5D90709F45FC020
:103A1000CC3CDC4509F460C030C0C23DFCE5DF07AA
:103A200009F46FC088F4CF3C9CE5D90709F460C065
:103A300008F45CC0C03DFCE5DF0709F45CC0C13D93
:103A4000DC4509F45BC019C0C53D9CE5D90709F404
:103A500060C050F4C33DFCE5DF0709F455C0C43D28
:103A6000DC4509F454C009C0C63D9CE5D90709F4FA
:103A700055C0CE35DD4509F454C011E052C00E9456
:103A8000DC1B4FC04EEC5BE161EC7BE104C041EC20
:103A90005BE16EEC7BE10E94AC1C43C041E159E16B
:103AA00064E079E1F8CF44E059E161E179E1F3CFF5
:103AB0004FE259E160E279E1EECF40E259E16FE295
:103AC00079E1E9CF4DE459E16EE379E1E4CF4EE3EA
:103AD00059E16DE479E1DFCF46EA57E16FE877E13C
:103AE000DACF4FE857E166EA77E1D5CF81E017C03A
:103AF00065E082E010C068E086E00DC06EE089E01D
:103B00000AC064E18FE007C067E185E104C088E195
:103B100006C062E289E10E94B21C03C083E20E94F7
:103B2000D11B812FDF91CF911F9108950F931F9388
:103B3000CF93DF938C01EB018091AE01811105C021
:103B40000E94F21F81E08093AE01AE01440F551F29
:103B50004C0F5D1F24E630E0B80180EBDF91CF9180
:103B60001F910F910C94A520CF93DF93EC01FB01E3
:103B70008281882309F43CC1C430FDE5DF0760F48D
:103B8000CB3F9CE5D90788F49E0122503C45243167
:103B9000310508F02EC109C0C236EDE5DE0729F077
:103BA000C63AFDE5DF0709F024C10E94FE0E90939E
:103BB000520280935102C1318CE5D80709F4C6C086
:103BC00008F042C0C930ECE5DE0709F49BC000F5FF
:103BD000C5308CE5D80709F485C078F4C330ECE52E
:103BE000DE0709F478C008F07AC0C230DC4509F07D
:103BF000F5C0809151028160EFC0C7309CE5D907C4
:103C000009F478C008F07AC0809151028061E4C064
:103C1000CD30FCE5DF0709F487C058F4CB309CE5D4
:103C2000D90709F479C008F07BC0809151028860FF
:103C30006FC0CF30FCE5DF0709F480C008F082C018
:103C400080915102877FC8C0CE3F9CE5D90709F417
:103C500071C000F5C531FCE5DF0709F485C068F4E3
:103C6000C3319CE5D90709F475C008F095C00E94DE
:103C7000AD08809151028F77AFC0CC3FFCE5DF07E4
:103C8000A9F108F054C0CB3FDC4509F0A7C08091F2
:103C9000520240C0C230EDE5DE0709F489C058F495
:103CA000C1158DE5D80709F45AC008F069C08091A4
:103CB000520282602FC0C236EDE5DE0709F47CC0F7
:103CC000C63AFDE5DF0709F481C0C330DD4509F0E0
:103CD00085C080E06EC08091510282607DC080917D
:103CE000510216C080915102886076C080915202C4
:103CF00082604FC08091510280626EC080915102FB
:103D000080646AC00E94AD0880915102806864C0DE
:103D1000846062C081603DC0809151028E7F5CC032
:103D2000809151028D7F58C08091510216C08091C0
:103D3000520218C0809152028D7F2BC08091510297
:103D40008F7E4AC0809151028F7D46C08091510282
:103D50008F7B42C080915102877F8B7F3DC08091D5
:103D600052028D7F8E7F15C08091510282FB2227E7
:103D700020F991E0922790FB82F990FB83F92CC007
:103D800080915202982F909591708E7F892B90FB95
:103D900081F98093520222C00E94AD0880915102A5
:103DA00087FB222720F991E0922790FB87F914C026
:103DB00081E00E94950F12C08091510284FB22275E
:103DC00020F991E0922790FB84F906C0809151027E
:103DD000982F909590FB80F9809351028091510229
:103DE000909152020E940F0F0E94AD0880E001C026
:103DF00081E0DF91CF910895CF93DF9386319C4589
:103E000041F5EB010E94020E982F8A8120916200F9
:103E100030916300882379F09A7A81E009F480E098
:103E20008093AF01911102C069E201C065E3C9014D
:103E30000E9468210AC08091AF01811102C069E22D
:103E400001C065E3C9010E946A210E94440E80E01E
:103E500001C081E0DF91CF9108950F931F93CF931D
:103E6000DF93C42FD22FFC0182818823C9F04093B5
:103E7000B2010E94A4219093B1018093B00180E22D
:103E80008C0F883008F057C0C77081E001C0880FE0
:103E9000CA95EAF7DF91CF911F910F910C940A0612
:103EA0008091B201481330C08091B0019091B1016E
:103EB0000E94BC21883C910538F510E21D0FCD17FA
:103EC000B9F080E28C0F883040F4C77081E001C007
:103ED000880FCA95EAF70E941106183028F581E08C
:103EE0009D2F977001C0880F9A95EAF70E940A06E5
:103EF000802F0E9401061830F0F4D77081E001C0D5
:103F0000880FDA95EAF70AC080E28C0F883098F4BF
:103F1000C77081E001C0880FCA95EAF7DF91CF91A1
:103F20001F910F910C941106802FDF91CF911F915B
:103F30000F910C940106DF91CF911F910F9108957D
:103F40000F939C01CB01243F4CE5340731F188F4F9
:103F5000293DFCE53F07D9F02A3D4CE5340779F1CE
:103F6000283D3C45A9F506E221EE41EE68ED7CE5F1
:103F70002BC0263FFCE53F07E1F0A8F0273F3C457A
:103F800039F507E225EE46EE67EF7CE51DC007E256
:103F900025EE45EE69ED7CE517C006E221EE40EE28
:103FA00064EF7CE511C007E225EE44EE65EF7CE5A9
:103FB0000BC006E221EE42EE66EF7CE505C008E2AA
:103FC00021E045EE6AED7CE50E942D1F80E008C0EF
:103FD000FC018281882319F01092B20101C081E0B6
:103FE0000F91089511B887E080B985B3836085BBD0
:103FF00086B7846086BF86B7816086BF86B78064D7
:1040000086BF08959F92AF92BF92CF92DF92EF92B8
:10401000FF920F931F93CF93DF93B82EEB010E9473
:10402000A4216C01C431D10558F0CF3F8FEFD807E0
:1040300059F0CE0164E170E00E9411257B0107C0B8
:10404000EE24E394F12C03C025E0E22EF12C84E869
:10405000A82E94EA992E16BE96BE0E94A4218C0129
:1040600006B607FC08C00E94A421801B910B8E1588
:104070009F05B0F324C081B1887F883039F081B1C9
:10408000887F803119F00FEF1FEF1BC0B3B8A6BEB9
:104090000E94A4218C0106B607FC08C00E94A4213E
:1040A000801B910B8E159F05B0F309C081B1887FED
:1040B000883111F0803439F700E010E00DC00EEFC8
:1040C0001FEFCF3F8FEFD80731F2C6010E94BC210E
:1040D0008C179D0708F4BFCFC801DF91CF911F91C6
:1040E0000F91FF90EF90DF90CF90BF90AF909F9097
:1040F00008950F931F93CF93DF93EB0183B984E867
:1041000086BF0E94A4218C0106B607FC0EC0CF3FDB
:104110008FEFD807C9F30E94A421801B910B8C1745
:104120009D0790F38EEF9FEF0BC021B1287F81E0B8
:1041300090E0283211F480E090E09195819591090A
:10414000DF91CF911F910F910895CF92DF92EF925F
:10415000FF920F931F93CF93DF936B018A01790135
:10416000B9010E940220E6010C0D1D1DC017D107E8
:1041700059F424E926BFDF91CF911F910F91FF9051
:10418000EF90DF90CF90089597FDF3CFB70189911D
:104190000E947920EBCF90931F0180931E01089518
:1041A0009093B8018093B7010895E091B701F09121
:1041B000B801309721F00190F081E02D099480E062
:1041C0000895E091B701F091B801309721F0028095
:1041D000F381E02D09940895E091B701F091B801C1
:1041E000309739F022E0DC012C930480F581E02D3A
:1041F000099408952091B5013091B6012817390727
:1042000071F09093B6018093B501E091B701F09100
:10421000B801309721F00680F781E02D09940895C8
:104220002091B3013091B4012817390771F09093B0
:10423000B4018093B301E091B701F091B8013097D8
:1042400021F00084F185E02D09940895FC01329657
:1042500097E080E0915029F021912223D9F38F5FDC
:10426000F9CF0895662349F0FC0132960896219112
:10427000621729F0E817F907D1F780E0089581E087
:1042800008959C01FC0132969FEF80E04191461712
:1042900089F09F3F19F4411101C0982F8F5F86303C
:1042A000A9F79F3F39F0F901E90FF11D97FDFA9544
:1042B0006283089508959C012A5F3F4FFC0142816B
:1042C000461301C01282019682179307B9F7089529
:1042D0000C9441210C945B21029626E0FC01119282
:1042E0002A95E9F7089508950C9473210C9474218C
:1042F0000C9473210C9473210C947321CF930E941E
:104300007A210E947B130E947821C0E08C2F0E94AA
:10431000AE12811104C0CF5FC430C1F701C081E08B
:10432000CF91089508958091BB0181110C945D0493
:1043300008950E94AD080C9461048BE083BF8BEB61
:104340008CBF82E089BF08952FB7F89480917502E1
:1043500090917602A0917702B09178022FBF0895D4
:104360002FB7F89460917502709176028091770270
:10437000909178022FBF08959C014FB7F8948091D7
:10438000750290917602A0917702B09178024FBFAA
:10439000821B930B089578941F920F920FB60F9281
:1043A00011248F939F93AF93BF9380917502909147
:1043B0007602A0917702B09178020196A11DB11DFD
:1043C0008093750290937602A0937702B09378025F
:1043D000BF91AF919F918F910F900FBE0F901F9043
:1043E000189560E081E090E00E94EF259CE088E174
:1043F0000FB6F894A89581BD0FBE91BDFFCF0E9466
:10440000A4219093BA018093B90108950E94E824F1
:104410008B9A80E0815041F0A895E7EBFBE0319763
:10442000F1F700C00000F6CF8B98789408950E94B1
:104430000B230E94D0202FEB84ED91E0215080408F
:104440009040E1F700C0000008958091A002882309
:1044500089F01092A0020E94A4219093BA01809347
:10446000B9018091BB018823D1F11092BB010E9458
:10447000992111C08091BB01811111C08091B901B6
:104480009091BA010E94BC21069728F081E08093A8
:10449000BB010E9493218091BB01882301F10E94FE
:1044A00093210E947E21882339F1F89421B3939AB5
:1044B000822F8C6081BB92B38CE0982792BB3FE542
:1044C0004AEE90E0315040409040E1F700C00000DB
:1044D00092B3892782BB21BB9398789408950E9458
:1044E000F1238091A602882329F08091840284FD23
:1044F0000E9467100C94B222089580915002089592
:1045000008959091C101981307C02091BF01309187
:10451000C00126173707A9F08093C1017093C0012D
:104520006093BF018093BC017093BE016093BD0195
:104530008091BD0284FF05C063E08CEB91E00C9498
:10454000ED230895BC0184E00C948122BC0183E03A
:104550000C9481222091BD0224FF03C066E00C94DC
:10456000ED230895CF93DF93CAE0D0E080918402D9
:1045700084FF18C08091CD019091CE019817E1F091
:1045800028E0829FC001112468E081539E4F0E9461
:10459000E9238091CD0190E001968F709927809357
:1045A000CD010AC00E94F12387EB9BE00197F1F750
:1045B00000C000002197D1F6DF91CF910895CF93ED
:1045C000DF93EC01A091CE01B0E0CD0101968F7098
:1045D00099272091CD01281779F093E0AA0FBB1FEE
:1045E0009A95E1F7A153BE4F98E0FE0101900D921C
:1045F0009A95E1F78093CE010E94F1230E94B222A6
:1046000088E0FE01A5ECB1E001900D928A95E1F7FA
:10461000DF91CF9108958FE790E00895FC018081AC
:1046200080768032A1F58181813061F48481958129
:10463000892B69F585EC91E09093A2028093A10209
:1046400088E00895823041F48FE492E09093A202D2
:104650008093A10281E008958A3021F483818093C0
:104660004F0215C0893099F482819381811592405F
:1046700081F484819581892B61F481E08093C40168
:10468000868197819093C3018093C20102C080E02C
:1046900008958FEF08952091C2013091C301232B1B
:1046A00071F02091C401213051F4FC01808180938C
:1046B00050021092C3011092C20181E008958FEF61
:1046C00008950895FC0193819330D9F068F49130F6
:1046D00081F0923009F059C083EE92E09093A202EB
:1046E0008093A1028BE30895913249F19232B9F19E
:1046F0004CC08EE193E09093A2028093A10282E1EC
:1047000008958281813099F050F08230F1F580E394
:1047100093E09093A2028093A1028EE0089588E531
:1047200093E09093A2028093A10284E0089580E434
:1047300093E09093A2028093A10286E10895828182
:10474000882329F0813009F58EE093E002C085EFDF
:1047500092E09093A2028093A10289E0089584815F
:104760009581009751F0019781F48CE593E0909347
:10477000A2028093A1028BE7089587ED93E09093C6
:10478000A2028093A10280E4089580E008951F931F
:10479000CF93DF93162FEA01288124FF05C03981CA
:1047A00028E82327298302C02AE52883212FFC013A
:1047B000CE010296DC0131913D9321501216DCF3BB
:1047C000612F0E9440021C5F1883DF91CF911F91DF
:1047D000089544E852E00C94C7234DEB52E00C944A
:1047E000C723CF93DF936091A302635067FD93C00B
:1047F00080919F02CCE0D0E0C81BD109C955DD4FA4
:1048000080919E02803120F4CE010E94612381C0FC
:104810008D3209F06EC0683009F07BC083EC809364
:1048200079028AE580938C0010929D0288818076BF
:1048300021F0CE010E940E2349C09A81109282027B
:104840008981811106C01092830222E832E082E061
:1048500038C0853019F49093A40230C08630A1F49A
:104860008B81813041F0823031F0833021F0813210
:1048700011F0823221F4CE010E94622301C080E057
:1048800090E490939D0222C0883089F0893019F419
:104890009093A60213C08A3069F08B3079F48BE4D0
:1048A000809385028093BE028093910207C026EA1E
:1048B00032E002C022E832E081E003C022E832E0C8
:1048C00080E03093A2022093A10209C08F3F39F407
:1048D000988197FD8E8190E890939D0207C09F81FB
:1048E000911104C09E81981708F4892F80938B0042
:1048F00010C080919D0287FF0CC0CE010E944B2307
:104900008F3F21F48EE180938C0003C081111092BF
:104910008B001092A30280918C0084FF4CC0809188
:104920008B008F3F09F447C0C82F893008F0C8E0DA
:104930008C1B80938B009091790288E88927809363
:104940007902CC2359F18091A1029091A202209189
:104950009D0226FF12C0A9E7B2E02C2FAC014957F7
:104960005240FA01EA0FFB1FE4911196EC93119764
:10497000215011962111F5CF08C0EAE7F2E0DC01E1
:104980002C2F3D9131932150E1F701962FEF2C0F01
:10499000820F911D9093A2028093A1026C2F8AE74F
:1049A00092E00E944002CC5FCC3019F08FEF8093F0
:1049B0008B00C0938C0084E190B39C7031F48150E3
:1049C000D9F71092A40210929C02DF91CF91089522
:1049D000CF93DF9385B7886085BF8BB780688BBF27
:1049E000C4E8D2E08BE48983ADEBB2E011968C93FE
:1049F0001197E0E9F2E081838AE588838C938083D4
:104A0000DF91CF91089587FB082E062687FD8195BB
:104A100067FD61950E9492250EF4919507FC8195A2
:104A20000895AA1BBB1B51E107C0AA1FBB1FA617F5
:104A3000B70710F0A61BB70B881F991F5A95A9F747
:104A400080959095BC01CD01089597FB072E16F433
:104A5000009407D077FD09D00E94112507FC05D0EE
:104A60003EF4909581959F4F0895709561957F4F85
:104A70000895A1E21A2EAA1BBB1BFD010DC0AA1F9F
:104A8000BB1FEE1FFF1FA217B307E407F50720F0B7
:104A9000A21BB30BE40BF50B661F771F881F991F32
:104AA0001A9469F760957095809590959B01AC017B
:104AB000BD01CF010895EE0FFF1F0590F491E02D89
:104AC00009940E946925332312F48A1B9B0B0C94D2
:104AD0007A25A29FB001B39FC001A39F700D811DD5
:104AE0001124911DB29F700D811D1124911D0895F7
:104AF0000E946925B7FF0895821B930B08950E94B9
:104B00006925A59F900DB49F900DA49F800D911DC8
:104B100011240895B7FF0C947F250E947F25821BE6
:104B2000930B0895991B79E004C0991F961708F01C
:104B3000961B881F7A95C9F780950895FC0141500E
:104B4000504030F001900616D1F73197CF0108950B
:104B5000882799270895FB01DC0104C08D910190FD
:104B6000801921F441505040C8F7881B990B0895D3
:104B7000E199FECF9FBB8EBBE09A99278DB3089534
:104B8000A6E1B0E044E050E00C94FE25A8E1B0E0DE
:104B900042E050E00C94FE25262FE199FECF9FBB0A
:104BA0008EBBE09A01970DB2021631F02DBB0FB605
:104BB000F894E29AE19A0FBE08950396272F0E9477
:104BC000CD250E94CC25252F0E94CD25242F0C9485
:104BD000CD250196272F0E94CD250C94CC25262F7C
:104BE000E199FECF9FBB8EBB2DBB0FB6F894E29A26
:104BF000E19A0FBE01960895DC01CB01FC01E19919
:104C0000FECF06C0FFBBEEBBE09A31960DB20D920F
:0C4C100041505040B8F70895F894FFCFD1
:104C1C00C8007B01280850011E0A14010101020082
:104C2C000700070701191A1B1C1D1E1F2021227DBE
:104C3C0022DF22AA22A622A2228022FF5AE200E927
:104C4C0000EA00B500B600B700CD008301CC008AA5
:104C5C00019201940121022302240225022602273B
:104C6C00022A02B300B4006F007000818283E2005C
:104C7C00E900EA00B500B600B700CD008301CC0016
:104C8C008A019201940121022302240225022602A8
:104C9C0027022A02B300B4006F0070008182836087
:104CAC0061626364659091929300010202020206B4
:104CBC0006060909090909090F0F0F0F0F0F151522
:0E4CCC0015181919191919191919191923246C
:00000001FF
